:020000040000FA
:1000000018308A00AE2D0000FF00030E8301A1000E
:100010000A08A0008A010408A2007708A300780853
:10002000A4007908A5007A08A6007B08A70083131E
:1000300083128C308400001C1F280C1832282208E0
:1000400084002308F7002408F8002508F900260892
:10005000FA002708FB0020088A00210E8300FF0E0B
:100060007F0E09008A110A1241280A108A100A110B
:10007000820700340034103430348A3400340034C1
:100080002D34061D452806114628061564000C105F
:100090008A110A121F28871087160530F700F70B00
:1000A0004F280000000000348C1A5828640054289F
:1000B0008C1E58281A088316D4008312981C6628B0
:1000C0001A088316D40083121812181683165408BF
:1000D000F800831200342908073C031D74280730F8
:1000E0000C1E70289900B32805308316C200420800
:1000F000063C0319B2284208053C031DAC282930F0
:10010000C40083126F088316C100043083120C1ED2
:10011000872899006F080C1E8B2899008316C3014D
:1001200083126F08831643020318A628440884002C
:100130000008C50083120C1E9B28990083164408F2
:1001400084000008C106C40AC30A9028410883122B
:100150000C1EA82899008316831254207808831651
:10016000C2007728831200349030A9000130AA0021
:100170003930AB00831681138312861DC2280230EA
:10018000AC00C4280130AC000430EF006B20003418
:10019000E030840000080319DC280130F800F70182
:1001A000F70BD028F80BCF283030F700F70BD62804
:1001B00000000000800BCD2800349130A9000230EF
:1001C000EF006B202A08F700F7080319F828013020
:1001D00077020319FE28023077020319042903303D
:1001E000770203190A290630770203191029172903
:1001F00005308316990022309800192902308316A1
:10020000990022309800192905308316990026306C
:100210009800192900308316990022309800192976
:10022000013083169900263098001929831283160D
:1002300019290230E0008312C8208A110A16CB283F
:10024000F701F8018316540803105518F707F70C47
:10025000F80CD518F707F70CF80C5519F707F70C39
:10026000F80CD519F707F70CF80C551AF707F70C27
:10027000F80CD51AF707F70CF80C551BF707F70C15
:10028000F80CD51BF707F70CF80C831200349230EA
:10029000A9006F08413C031966290130AA008316A2
:1002A000BA013A083F3C031C642902303A07293E50
:1002B00084003A08D4000530D50083122021780844
:1002C00080008316BA0A51299D2983128316BA0128
:1002D0003A083F3C031C7F2901303A07293E84003D
:1002E0000008BC003A08D4000530D5008312202154
:1002F000780883163C02031D7F29BA0A68293A0848
:100300003F3C031C85290130862900308312AA0056
:100310008316BA013A083F3C031C9D2902303A0774
:10032000293E84003A08D4000530D50083122021EC
:10033000780880008316BA0A8A2942308312EF00B7
:100340006B208A110A16D3289530A9000508AA0047
:100350000608AB000708AC00053083169F00831227
:100360001F083839C1389F000030F8001F08C7390E
:1003700078049F001E30F700F70BBC2900001F1502
:100380001F19C0291E08AD000830F8001F08C73922
:1003900078049F001E30F700F70BCC2900001F15D2
:1003A0001F19D0291E08AE000630EF006B20003464
:1003B0006F08073C031DEF292A0883168500831266
:1003C0002B088316860083122C088316870083125D
:1003D0002D0885002E0886002F088700A4218A1189
:1003E0000A16DB282A088316BB002B30BC00BA0192
:1003F000023083126F0283163A0203182B2A3B083D
:10040000BB0ABD003C08BC0A84000008BE003D08D1
:10041000831203178D008F01831603133E08831286
:1004200003178C0083168C130C15831203130B080F
:10043000F7008B138316031755308D00AA308D00FB
:100440008C148C18212A0C117708831203138B0447
:100450008316BA0AF82907308312A9000130EF0089
:100460006B208A110A16EB282A088316BB002B3052
:10047000BC0083122B08EF008316BA0183126F08A9
:1004800083163A020318582A3C08BC0A84003B0829
:10049000BB0ABE00831203178D008F0183168C13D5
:1004A0000C1483120C08800083160313BA0A3E2A28
:1004B000E3308312A9000230EF076B208A110A167D
:1004C000F328E530A9000130AA000230EF006B20CC
:1004D0008A110A16FB28E730A9004630AA0002302C
:1004E000EF006B208A110A1603298712003480302E
:1004F0008316870581308704D93086050616DB30E0
:1005000085051B3085040515851686148312871111
:1005100007124B20752287140530F700F70B8E2A3F
:10052000000000004B20752287140530F700F70B00
:10053000972A000000000034831622081F3C031D88
:10054000C42AE2016208053C031CC32A83128715F2
:1005500003108316E00C0318B12A83120712B32A82
:100560008316831207160530F700F70BB52A000033
:10057000000087110530F700F70BBC2A00000000CF
:100580008316E20AA22AF82B6008E03E0318F82B33
:10059000203E8312FA2B0712871587110712871541
:1005A0008711071287158711071287158711071200
:1005B000871587110712871587118316F82B0716E1
:1005C000871587110712871587110712871587115D
:1005D00007128715871107128715871107128715CC
:1005E00087118316F82B07128715871107168715B1
:1005F00087110712871587110712871587110712B0
:10060000871587110712871587118316F82B071690
:100610008715871107168715871107128715871108
:10062000071287158711071287158711071287157B
:1006300087118316F82B0712871587110712871564
:10064000871107168715871107128715871107125B
:10065000871587110712871587118316F82B071640
:1006600087158711071287158711071687158711B8
:10067000071287158711071287158711071287152B
:1006800087118316F82B0712871587110716871510
:10069000871107168715871107128715871107120B
:1006A000871587110712871587118316F82B0716F0
:1006B0008715871107168715871107168715871164
:1006C00007128715871107128715871107128715DB
:1006D00087118316F82B07128715871107128715C4
:1006E00087110712871587110716871587110712BB
:1006F000871587110712871587118316F82B0716A0
:10070000871587110712871587110712871587111B
:100710000716871587110712871587110712871586
:1007200087118316F82B071687158711071687156B
:10073000871107128715871107168715871107126A
:10074000871587110712871587118316F82B071253
:1007500087158711071687158711071687158711C3
:100760000716871587110712871587110712871536
:1007700087118316F82B071687158711071687151B
:100780008711071687158711071287158711071616
:10079000871587110712871587118316F82B071203
:1007A000871587110712871587110712871587117B
:1007B00007168715871107168715871107128715E2
:1007C00087118316F82B07168715871107168715CB
:1007D00087110716871587110716871587110716C2
:1007E000871587110712871587118316F82B831633
:1007F0008312003400000A108A100A15023E031802
:100800008A0A8200CB2ADF2AF32A072B1B2B2F2BE5
:10081000432B572B6B2B7F2BF72B932BF72BF72B84
:10082000A72BF72BF72BF72BF72BF72BF72BF72B08
:10083000F72BBB2BCF2BF72BF72BF72BF72BF72B0C
:10084000F72BE32B01308316AA000230A500A3008A
:10085000A6012608A4000830A8000E30A9006430C4
:10086000A7000930B8000630E00083129C22003453
:100870008316A5012508A3006430A600A400083053
:10088000A8000E30A9001930B3006430B400033062
:10089000B5001F305F02FF3E0318592C013E831242
:1008A0005D2C64308316E0008312C8208316592C17
:1008B000831683128A110A124C2E0A108A100A1506
:1008C0008207512C77222808FF3E03184F2E013E45
:1008D000502E83165D08DE00A101A0015E08A20073
:1008E000A901A701AA012030AC00AB01AE0007307E
:1008F000AD000130AF00B0010130B100B201B6016E
:100900003710B8012208F7001030220283120319B1
:10091000E62C123077020319F12C153077020319F7
:10092000FF2C1130770203190B2D133077020319B6
:10093000162D163077020319262D1C307702031965
:10094000322D1730770203193E2D1D30770203191F
:100950004A2D183077020319562D193077020319E2
:10096000612D1A30770203196D2D143077020319A7
:10097000792D043077020319912D1B30770203196A
:10098000A92D033077020319C12D0730770203190F
:10099000CC2D0B3077020319D82D0C3077020319B8
:1009A000E42D083077020319F02D0930770203197E
:1009B000022E053077020319142E06307702031930
:1009C000202E0A3077020319342E472E0830831662
:1009D000A500A300A6012608A4000830A800B801BD
:1009E0004D2E08308316A500A300A6012608A400FA
:1009F0000830A8000130B6000130B8004D2E0D308F
:100A00008316A500A300A6012608A4000830A800AC
:100A10000330B8004D2E04308316A500A300A601B4
:100A20002608A4001830A800B8014D2E0230831605
:100A3000A500A300A6012608A4001830A8001730BE
:100A4000A9000130B6000130B8004D2E08308316E1
:100A5000A500A300A6012608A4001830A8000330B2
:100A6000B8004D2E03308316A300A4010630A50064
:100A7000A6010830A8000430B8004D2E08308316B7
:100A8000A500A300A6012608A4000830A800053090
:100A9000B8004D2E08308316A500A300A601260835
:100AA000A4000830A8000830B8004D2E143083167A
:100AB000A500A300A6012608A4000830A800B801DC
:100AC0004D2E08308316A500A300A6012608A40019
:100AD0000830A8000330B8004D2E04308316A5005E
:100AE000A300A6012608A4001830A8000330B8000F
:100AF0004D2E01308316A500A300A6012608A400F0
:100B00000830A8000E30A9000230AF000130B0005C
:100B10000230B1000130B2000330B6000230B8003C
:100B20004D2E02308316A500A300A6012608A400BE
:100B30001830A8001730A9000430AF000330B0000F
:100B40000430B1000330B2000330B6000630B80004
:100B50004D2E01308316A500A300A6012608A4008F
:100B60001830A8001730A9000430AF000330B000DF
:100B70000430B1000330B2000330B6000730B800D3
:100B80004D2E01308316AC00AB01AE00FF30AD003E
:100B90008312222483164D2E02308316AC00AB0143
:100BA0000330AE00FF30AD008312222483164D2E99
:100BB00002308316AC00AB010330AE00FF30AD0055
:100BC0008312222483164D2E04308316AC00AB0111
:100BD0000730AE00FF30AD008312222483164D2E65
:100BE00003308316A300A4010630A500A601083037
:100BF000A8000430AF000330B0000330B60004306A
:100C0000B8004D2E03308316A300A4010630A500C2
:100C1000A6010830A8000830AF000730B00003304C
:100C2000B6000430B8004D2E02308316AC00AB0184
:100C30000330AE00FF30AD008312222483164D2E08
:100C400008308316AC00AB010F30AE00FF30AD00B2
:100C50000430AF000330B0000430B1000330B20004
:100C60008312222483164D2E02308316A500A30082
:100C7000A6012608A4001830A8000E30A900643090
:100C8000A7000330B6000230B8004D2E8312831641
:100C90005E08DF008312382C831683124F2E003437
:100CA0000A108A140A158207692C2A088316BA00CA
:100CB0003A08E0398312A80083163A08DD0083124F
:100CC00062240730A9000130EF006B208A110A1658
:100CD0000B2983163A1083122A080139003A0319A6
:100CE000782E6F08023C031D782E83163A14831267
:100CF000003083163A180130BB00BC0083124B2031
:100D000007110C3097000030F800043892001530BD
:100D100083169200BC080319952E0B3083129500A0
:100D20001708CF3997009B2E831606308312950043
:100D30001708CF3997004B2004308316BB00AF3023
:100D4000E0008312C8208316BB0B9F2E073083124E
:100D5000A9000130EF006B208A110A161329071130
:100D6000970197014B200730A9000130EF006B205D
:100D70008A110A161B29831622081F3C031D062F01
:100D80008312871507160530F700F70BC52E0000F4
:100D9000000087110530F700F70BCC2E0000000093
:100DA0008316E20162080D3C031CF42E83128715A2
:100DB00003108316E10CE00C0318E22E83120712D5
:100DC000E42E8316831207160530F700F70BE62E84
:100DD0000000000087110530F700F70BED2E000032
:100DE00000008316E20AD22E8312871507160530FB
:100DF000F700F70BF92E0000000087110530F7000F
:100E0000F70B002F00000000262F83168312871592
:100E1000071687118316E20162080D3C031C222F7E
:100E20008312871503108316E10CE00C03181C2FA6
:100E3000831207121E2F831683120716871183163B
:100E4000E20A0C2F83128715071687110000640031
:100E5000003483165D08E00083129C2283165F082D
:100E6000E1005E08E0008312BB26003483162A08E6
:100E70000139003A03194C2F2D085B02031D4C2F3A
:100E80002E085C02031D4C2F8312772283165C0808
:100E9000A1005B08A000832F5C082102031C562FD1
:100EA000031D5E2F20085B02031C5E2F5C081F3CA5
:100EB0000318832F21081F3C031C832F5C081F3C51
:100EC000031C712F2208DD00831262240230831676
:100ED000DD003F30DF00FF30DE0083122927822F44
:100EE00083162208DD00831262248316DD013F3061
:100EF000DF00FF30DE008312292720308316A10097
:100F0000A0018312831621085C02031C962F031D87
:100F10008D2F5B0820020318962F0630E000831205
:100F20009C228316A00A0319A10A832F831200347E
:100F300083163C08FD3E0318B92F033E8312D52FBC
:100F400009308316BC002030DC00DB018312362719
:100F50008316B92F0B308316BC00B92F1F308316B0
:100F6000BC002030DC00DB01831236278316B92F4A
:100F700083163C08E00083129C2204308316E000B4
:100F80008312C82083163C081F3C0319D12F083058
:100F9000E00083129C2202308316E0008312C820F6
:100FA000831683128A150A12AA2C0A148A140A15A7
:100FB0008207A02FAA2FAE2FD6308400FC308005E8
:100FC000800C800C00080319E92FE72F0000800B2C
:100FD000E62F00348A15D5208A11013083162007A8
:100FE000D6002108D7000318D70A5708DC00560896
:100FF000DB00831236270034EE060034EE060034A0
:1010000083163C08FD3E03183A28033E83123E280F
:101010008316E0018A1183129C228A153F308316C1
:10102000E100FF30E0008A118312BB268A150930E7
:101030008316E0008A1183129C228A1506308316DB
:10104000E0008A118312C8208A158316BC08031990
:101050003A280B308316E0008A1183129C228A15ED
:1010600006308316E0008A118312C8208A15831681
:101070003A28831683128A150A12442D0A108A1000
:101080000A11820708282928082883165908E00031
:101090008A1183129C228A15831607165A08DB00D0
:1010A00022081F3C031D7A28DC015C080F3C031C4E
:1010B0007928831287150000071A60280310612819
:1010C000031483165B088400840A800C8403800C5C
:1010D0000530F700F70B6A28000000008312871123
:1010E0000530F700F70B7228000000008316DC0AB9
:1010F00055289328DC015C080F3C031C93288312BD
:1011000087150000071A8628031087280314831602
:101110005B088400840A800C8403800C831287118E
:101120008316DC0A7B285B088400013084070310E7
:10113000800C8403800C5B0884000008F700840A9C
:1011400000083F39FA00770884038000840A7A088F
:1011500080008403000064000712831200348316A9
:10116000C801470848020318D3284508FA00440874
:10117000C40A0319C50AC9007A08CA00DC00490874
:10118000DB008A11831236278A1583164808460722
:10119000C9000430D9004908DA0083124520023022
:1011A0008316C807B1288312003483162808E0008C
:1011B0008A1183129C228A1583162308E0008A1163
:1011C0008312C8208A1583162408D6008A11831238
:1011D000DC278A158316A9080319F5282908E000D9
:1011E0008A1183129C228A1583162708D6008A1139
:1011F0008312DC278A150034831650080739D5007E
:101200002208123C031D3229F830D0053F30D105A9
:10121000D40155085402031832295108FA00500825
:10122000D00A0319D10AD9007A08DA00DC0059087B
:10123000DB008A11831236278A1504308316D90001
:10124000D630DA008312452002308316DD005708BD
:10125000DF005608DE008A11831229278A158316BB
:10126000D40A0929D4015308540203185F295108EC
:10127000FA005008D00A0319D10AD9007A08DA0016
:10128000DC005908DB008A11831236278A15831681
:101290005208D20AD20A8400840A0008DA008403C1
:1012A0000008D9000230DD005A08DF005908DE00CE
:1012B0008A11831229278A158316D40A3329220812
:1012C000123C031D972951081F3C03186A2904305A
:1012D000D8006C290830D8005508D30758085302A5
:1012E000031897295108FA005008D00A0319D10AA7
:1012F000D9007A08DA00DC005908DB008A11831271
:1013000036278A1504308316D900D630DA008312C6
:10131000452002308316DD005708DF005608DE0046
:101320008A11831229278A158316D30A6E298312FC
:1013300000348316D5010130540255020318C72921
:101340005308D30AD30A8400840A0008D700840310
:101350000008D6000230DD005708DF005608DE0026
:101360008A11831229278A15013083162007D60097
:101370002108D7000318D70A5708DC005608DB00FD
:101380008A11831236278A158316D50A9B2953089A
:101390008400840A0008D70084030008D6000230C5
:1013A000DD005708DF005608DE008A118312292766
:1013B0008A158A11EA278A15003483163608FB3EFF
:1013C0000318A82B053E8312AA2B83164608CA00D1
:1013D0004508C9004708CB004808CC004B08CE00A0
:1013E0004A08DC004908DB008A11831236278A1577
:1013F0008316CD014C084D0203181C2A01304D07FD
:101400004E0784000008D0004E084D0784000008F5
:10141000D1005008D2000230DD005008DF00510832
:10142000DE008A11831229278A158A11EA278A1574
:1014300002308316CD07FA29A82B83164608CA0066
:101440004508C9004708CB004808CC004B08CF002E
:101450000310CC0C49080739F7004A080039FA0094
:101460007708083CCE004C020318382A4C08CE00FE
:101470004A081F3C03187F2AFF3A031D432A4908E4
:10148000033C03187F2ACD014C084D0203187E2A25
:101490004A08FA004908C90A0319CA0AD0007A089A
:1014A000D100DC005008DB008A11831236278A1530
:1014B00083164F08CF0ACF0A8400840A0008D1009F
:1014C00084030008D0000230DD005108DF0050081E
:1014D000DE008A11831229278A1508308316E0005E
:1014E0008A1183129C228A1506308316E0008A1125
:1014F0008312C8208A158316CD0A442ABE2A4A08B8
:10150000D1004908D0004B08D2004E08D300831206
:10151000FC208A11EA278A1583164E08CC02031094
:101520004E0DF700CF070830CD004D084C02031CCC
:10153000AC2A2108D1002008D0004F08D200083082
:10154000D3008312FC208A11EA278A1510308316F3
:10155000CF070830CD07952A0730CC050319BE2ADE
:101560002108D1002008D0004F08D2004C08D30039
:101570008312FC208A11EA278A158316A82B83166A
:101580004608CA004508C9004708CB004808CC00F7
:101590004B08D0000310CC0C4A081F3C0318D52A76
:1015A0003108D1003208D200D92A2F08D1003008E2
:1015B000D20049085205CF004A08DC004908DB0088
:1015C0008A11831236278A158316CF080319FD2A3C
:1015D0004F085102CE004C020318F02A4C08CE00EE
:1015E0005008D3004E08D4008312992183164E0868
:1015F000CC0203104E0DF700D0074C085205CD0069
:101600005208FF3ACC05CC080319142B5008D3001C
:101610005108D4008312992103108316510DF7004D
:10162000D0075108CC02032BCD0803191E2B5008FC
:10163000D3004D08D400831299218316A82B83165A
:101640004608CA004508C9004708CB004808CC0036
:101650004B08CD000310CC0CCC080319A62B4A086C
:10166000FA004908C90A0319CA0AD3007A08D40043
:10167000DC005308DB008A11831236278A15831693
:101680004D08CD0ACD0A8400840A0008FA008403BC
:101690000008CE007A08CF004A081F3C03185A2BD6
:1016A000FF3A031D572B4908073C03185A2B3408EF
:1016B000D200922B3308D2000230DD004F08DF0049
:1016C0004E08DE008A11831229278A15D52004309E
:1016D0008316D900D030DA00831245208316D20356
:1016E00003197A2B4E085002031D5C2B4F08510240
:1016F000031D5C2B4E085002031D912B4F08510215
:10170000031D912B52083302D3003508D40053082F
:10171000D5008A11831220218A1578088316D200F9
:10172000922BA62B5208D203003A0319A42B0230A5
:10173000DD004F08DF004E08DE008A1183122927E2
:101740008A15D5208316922BCC032C2BA82B83161D
:10175000831200340A148A140A118207E5291D2A0B
:10176000A72BBF2A1F2B83163C08FD3E0318F82B1E
:10177000033E8312FC2B20308316C5000730C400C3
:10178000C030C6000230C7008312AF200930831674
:10179000E0008A1183129C228A1508308316E0002B
:1017A0008A118312C8208A15FF308316C0040F30B7
:1017B000C1042030C6000730C500C030C700023069
:1017C000C8008312DD218316BC080319F82B0B30E7
:1017D0008316E0008A1183129C228A150830831632
:1017E000E0008A118312C8208A158316F82B83160D
:1017F00083128A150A124B2D0A108A100A158207C5
:10180000BB2BE72BBB2B83163C08FD3E0318272C74
:10181000033E8312302C20308316DC000930DB00BD
:101820008A11831236278A1509308316E0008A113F
:1018300083129C228A158316272C0B308316E00016
:101840008A1183129C228A158316272C8316063050
:10185000E0008A118312C8208A158A150A12552EB3
:101860000A108A100A158207142C1D2C0B2C8316C3
:101870003808F63E03187E2E0A3E8312822E831607
:101880003B08BC003C08F700F708831203194D2CF5
:10189000013077020319512C562C02308316BC00FC
:1018A000582C03308316BC00582C83128316BC01BD
:1018B0003C08E0008A1183129C228A153F3083166F
:1018C000E100FF30E0008A118312BB268A158316DF
:1018D000BC08031D792CBD013D08063C031C792C76
:1018E0000630E0008A1183129C228A158316BD0AF5
:1018F0006C2C0130E0008A1183129C228A1507307B
:101900008316E0008A1183129C228A150830831600
:10191000E0008A1183129C228A1508308316E000A9
:101920008A118312C8208A1501308316E0008A11BB
:1019300083129C228A1507308316E0008A118312D5
:101940009C228A1583167E2E83163B08BC008A11C2
:101950008312982F8A1583167E2E20308316DC0082
:10196000DB018A11831236278A1509308316E000BD
:101970008A1183129C228A151E308316E0008A1178
:101980008312C8208A1583167E2E83163B08BC005E
:101990003C08F700F70883120319D32C01307702B3
:1019A0000319D72CDC2C09308316BE00DD2C0B303C
:1019B0008316BE00DD2C83128316E0018A11831288
:1019C0009C228A153F308316E100FF30E0008A1127
:1019D0008312BB268A158316BD013D08063C031CF5
:1019E000FA2C0630E0008A1183129C228A15831695
:1019F000BD0AED2C3C08023C0319142D3E08E00002
:101A00008A1183129C228A1518308316E0008A11ED
:101A100083129C228A1505308316E0008A118312F6
:101A2000C8208A153D2D83160130E0008A118312EB
:101A30009C228A1507308316E0008A1183129C22AB
:101A40008A1508308316E0008A1183129C228A15B9
:101A50000D308316E0008A118312C8208A150130E8
:101A60008316E0008A1183129C228A1507308316A0
:101A7000E0008A1183129C228A1583167E2E83161B
:101A80003B08BC008312002883167E2E83163B0879
:101A9000BC008312B32B83167E2E83163B08BC003A
:101AA000BC080319572D3C08023C031DB82DDC016E
:101AB000DB018A11831236278A1502308316DD0076
:101AC0003F30DF00FF30DE008A11831229278A159C
:101AD0008316BE01BD01BE08031D9B2D3D087F3C42
:101AE000031C9B2D0830E0008A1183129C228A156A
:101AF00002308316E0008A118312C8208A1517303D
:101B00008316E0008A1183129C228A1520308316E6
:101B10002007BF002108C0000318C00A4008DC00ED
:101B20003F08DB008A11831236278A158316BD0A07
:101B30000319BE0A6B2D2030DC00DB018A118312F1
:101B400036278A1508308316E0008A1183129C22FA
:101B50008A1502308316E0008A118312C8208A1584
:101B600017308316E0008A1183129C228A1583168F
:101B70003C0BBB2DBF2D3C08023C031DFF2DDC019F
:101B8000DB018A11831236278A1503308316DD00A4
:101B9000DF01FF30DE008A11831229278A158316A0
:101BA000BE01BD013E08003C031CFF2D0830E000D3
:101BB0008A1183129C228A1502308316E0008A1152
:101BC0008312C8208A1517308316E0008A11831209
:101BD0009C228A15013083162007BF002108C0000F
:101BE0000318C00A4008DC003F08DB008A1183129A
:101BF00036278A158316BD0A0319BE0AD22D7E2EFA
:101C000083163B08BC000230BD001730BE002030F8
:101C1000DC00DB018A11831236278A1583163C0803
:101C2000F700F708831203191A2E013077020319FF
:101C3000252E312E09308316E0008A1183129C2252
:101C40008A1508308316BC00372E0B308316E0004F
:101C50008A1183129C228A1508308316BC00372E05
:101C600083121F308316BC000830BD00BE013C0843
:101C7000E0008A1183129C228A1583163D08E00039
:101C80008A118312C8208A158316BE0803194F2EA5
:101C90003E08E0008A1183129C228A1583167E2E4C
:101CA00083163B08BC008312032C83167E2E8316FA
:101CB0003B08BC002C08DC002B08DB008A118312D7
:101CC00036278A1502308316DD003F30DF00FF30F3
:101CD000DE008A11831229278A1509308316E00055
:101CE0008A1183129C228A150A308316E0008A1119
:101CF0008312C8208A1583167E2E831683128A15B6
:101D00000A129B2E0A108A140A1582073F2CA42C53
:101D1000AD2CC52C3F2D462D4D2D002E502E572E6F
:101D20002808FF3E03189C2E013EA12E83163A0878
:101D3000BB008312372C9C2E871107128A150A12BA
:101D4000AB2E0A108A140A158207962E2A088316CB
:101D5000BA008312902E0730A9000130EF008A11DB
:101D60006B208A158A110A1624292808FF3E0318B9
:101D7000C72E013ECC2E83164008C6003F08C50082
:101D80004308C7004408C8008312DD21C72E87110D
:101D900007128A150A12F22E0A108A140A158207EF
:101DA000BB2E8316BD0183122C088316BC00831240
:101DB0002B088316BB0083122A088316BA0004304E
:101DC00083126F028316BE003D08C2003C08C100AA
:101DD0003B08C0003A08BF002D30C3003E08C400D5
:101DE0008312B52E0730A9000130EF008A116B2055
:101DF0008A158A110A162E292808FF3E03180E2F6D
:101E0000013E132F83163F08C5003E08C400420858
:101E1000C6004308C7008312AF200E2F8711071298
:101E20008A150A123A2F0A148A140A158207022FF9
:101E30008316BD0183122C088316BC0083122B0865
:101E40008316BB0083122A088316BA0083122D085A
:101E5000EF0083163D08C1003C08C0003B08BF00EE
:101E60003A08BE002D30C20083126F088316C300EB
:101E70008312FC2EC430A9000430EF078A116B20B6
:101E80008A158A110A1638292808FF3E0318A32F3D
:101E9000013EA82F83163E08C2003D08C1003F083E
:101EA000C3004008C4004208DC004108DB008A117E
:101EB000831236278A158316C50144084502031884
:101EC000A12F4508430784000008C6000330DD0049
:101ED000DF014608DE008A11831229278A1583163E
:101EE0002808E0008A1183129C228A15831625088F
:101EF000E0008A118312C8208A1583162608D600AE
:101F00008A118312DC278A158316A90803198F2FDB
:101F10002908E0008A1183129C228A158316013059
:101F20002007C6002108C7000318C70A4708DC00BD
:101F30004608DB008A11831236278A158316C50AE4
:101F40005D2F8312A32F871107128A150A12C32F40
:101F50000A148A140A1582074A2F2B088316BB001D
:101F600083122A088316BA00033083126F02831685
:101F7000BC003B08BE003A08BD002C30BF003C0846
:101F8000C0008312442F0730A9000130EF008A11EE
:101F90006B208A158A110A1642292B088316BB006A
:101FA00083122A088316BA0083122C08EF008316C6
:101FB0003B08BD003A08BC002C30BE0083126F08FD
:101FC0008316BF000A168A11831200280A128A1586
:101FD000E230A9000330EF078A116B208A158A11BD
:101FE0000A164C2900308C1A0130F80000342908F8
:101FF0000C1EF82F99002908EE0600340034003436
:102000002808FF3E03183928013E3E2883163D0864
:10201000C1003C08C0003E08C2003F08C300C40124
:1020200043084402031837284108FA004008C00A50
:102030000319C10AC7007A08C800DC004708DB00A2
:102040000A12831236270A1605308316D900C530C6
:10205000DA000A128A15831245200A168A1183169D
:1020600044084207840045088000C40A10288312EF
:102070003928871107128A150A12E62F0A108A10CA
:102080000A11820706280A124B200A16D030A9002E
:10209000AA01AB01AC01AD010530EF000A126B20C3
:1020A0000A168A110A1654290A1275220A16D03005
:1020B000A9000130AA00AB01AC01AD010530EF0071
:1020C0000A126B200A168A110A165A290130831641
:1020D000B900BD012930BE00BD08031DBC280A128D
:1020E000831254200A1678088316BA003A08043C72
:1020F000031982280A12831254200A1678088316BC
:10210000BA0076280A12831254200A167808EF00C3
:102110008316BC00BB0183126F0883163B020318B1
:10212000A3283E08BF000A12831254200A16831601
:102130003F088400780880003E0884000008BC0640
:10214000BE0ABB0A8B280A12831254200A1678088A
:102150008316BC06031DB5280130BD00063083126E
:102160000C1EB0289900BA288316053083120C1E65
:10217000B728990083166C2883122908103C031D88
:10218000C5280A12B4200A165E292908113C031D2D
:10219000CD280A12DD280A165E292908123C031DE3
:1021A000D5280A1247290A165E292908143C031D5E
:1021B000DD280A12D8290A165E292908153C031DB4
:1021C000E5280A12A4210A165E292908173C031DD6
:1021D000ED280A12F2290A165E292908183C031D67
:1021E000F5280A12342A0A165E2929081A3C031D0A
:1021F000FD280A12612A0A165E2929081B3C031DC4
:1022000005290A126B2A0A165E292908413C031D7A
:102210000D290A12552E0A165E292908403C031D75
:1022200015290A12692E0A165E292908473C031D42
:102230001D290A12AF2E0A165E292908433C031DE8
:1022400027290A128A15A62E0A168A115E2929083C
:10225000423C031D31290A128A15D12E0A168A1111
:102260005E292908443C031D3B290A128A15182FB0
:102270000A168A115E292908453C031D45290A12C0
:102280008A15AD2F0A168A115E292908463C031DBE
:102290004F290A128A15CD2F0A168A115E2929089C
:1022A000503C031D552943285E292908513C031D34
:1022B0005B2954285E298316B901831283163908D5
:1022C000F80083128A150A16162E83166614640007
:1022D0008312071E7F29640083166508E503003A10
:1022E000031D7729661083127F297E2983164D30BE
:1022F000F700F70B792900000000831269290030EC
:10230000831666180130F8008312003483165D0DC1
:10231000DE00DE0DDE0DF830DE050716FF30E500CD
:10232000831265218316E001DF0160087102031C3E
:10233000A729031D9F295F087002031CA7290230EB
:10234000F700F70BA129DF0A0319E00A9529831288
:1023500087158316E001DF0160087102031CBF29A5
:10236000031DB6295F087002031CBF290630F70061
:10237000F70BB8290000DF0A0319E00AAC29831221
:10238000071AC4290310C52903148316E10DE20DB1
:10239000E30D07128312071283165D0BD529031074
:1023A000D90D031CD5290716EA295D08023C031D37
:1023B000E0290310D90DDA0D031CE0290716EA29DC
:1023C0005D08033C031DEA290310D90DDA0DDB0D6E
:1023D00003180716831287118316E001DF016008D6
:1023E0007102031C022A031DF9295F087002031CF5
:1023F000022A0630F700F70BFB290000DF0A031959
:10240000E00AEF290716DE0BA72907166108F70077
:102410006208F8006308F9006408FA0083120034C7
:102420000830F7000718122A8316D501F717282A53
:10243000F713282A03108312071803148316D50CE8
:102440007717282A7713F70B1A2A5508F800352A28
:102450007930F71B2130F800F80B2C2A000000001F
:10246000F71B182A771B222A1A2A83128A110A16A6
:102470002D2B08300C1E3A2A99008316510883121E
:102480000C1E402A9900003407100830F8000000A4
:1024900000000000F8175D2AF8138316D20C83128F
:1024A00003180714031C071078175D2A7813F80B1C
:1024B0004D2A000000000000071479308400840BCE
:1024C0005F2A00000000F81B4C2A781B562A8A114C
:1024D0000A16BB2BFF308316CF00D000D100D201EB
:1024E000E50183126521F8080319962A2808FF3EA2
:1024F0000318962A013EA12A8316DC01DB01403035
:10250000DA00D9010230DD008312862178081F39F4
:10251000FA007708F8007A08F9008316D201D10191
:102520007908D0007808CF008312962A83164F08C6
:10253000F7005008F8005108F9005208FA00831219
:1025400000340A108A140A1182077C2AFF3083168D
:10255000CB00CC00CD00CE01E50183126521F80847
:102560000319012B2808FF3E0318012B013EF42B11
:1025700083164708D0004608CF004708D200460817
:10258000D100FF30D300D4005108F70052081F39A2
:10259000FA005108D5007A08C038D600D701D80112
:1025A0005808DC005708DB005608DA005108D9004B
:1025B0000230DD00831286218316E5018312652136
:1025C000F8080319F42A8316DC01DB014030DA0035
:1025D000D9010230DD008312862177088316D300EB
:1025E00078081F39D400831283165308F800540862
:1025F000F900CE01CD017908CC007808CB00831218
:10260000012B8316CA080319CC2B4F104F18CC2B63
:10261000E50183126521F8080319102B8316CC2BD2
:10262000D0308316D1005214D21086108312861433
:1026300083160714741C212B51088400013080007C
:10264000562BD218562B640083120718352B83168D
:1026500051088400D4008312102A83165408840081
:1026600078088000D214552B83120A128A15F2279B
:102670000A168A11F8080319492B0A1254200A165F
:102680007808023C031D482B8316D2145210831283
:10269000542B8316E50183126521F8080319542B86
:1026A0008316D214521083128316212B0030521835
:1026B0000130F800F8080319C82B5008F700013062
:1026C000770283120319652BC12B01308316D100C9
:1026D00083123922D0308316D1005214D210D2186E
:1026E000AB2BE50183126521F8080319792B8316BA
:1026F000AB2B0A128A15F2270A168A11F808031959
:10270000A92B83165108D3000A12831254200A16EB
:10271000831653088400780880005108840000085C
:10272000083C031DA02B5108D3000A128312542029
:102730000A1683165308840078088000D214A82B48
:10274000510884000008023C031DA82BD21452102B
:10275000831283166F2B003052180130F800F808EE
:102760000319BD2B74105008D100861407105108AE
:10277000D2008312442AC02B831674144F14831280
:10278000C62B83165008D10083123922CA2B831618
:102790004F1483128316062B4B0FD52B4C0FD52BC2
:1027A0004D0FD52BCE080319DF2B4B0FEA2B4C0F07
:1027B000EA2BCD08031DEA2BCE08031DEA2B83125A
:1027C0006A227A088316CE007908CD007808CC00FA
:1027D0007708CB004B08F7004C08F8004D08F900CB
:1027E0004E08FA00831200340A148A140A11820770
:1027F000B82A0A124B200A1687150A1275220A16E1
:102800000230F700F70B022C000000008711FF30A8
:102810008316E500831265218316C901C801C7012B
:10282000C601CA018312A6220A124B200A16871576
:102830000A1275220A160230F700F70B1D2C000051
:10284000000087118316DC01DB014030DA00D9017A
:102850000230DD008312862178081F39FA007708DC
:10286000F8007A08F90000348316C401C501F101AB
:102870007330F000FF30E50083126521F80803197A
:10288000A22C8316DC01DB011030DA00D901023002
:10289000DD0083128621831607168312071A4E2C39
:1028A0008316C501C40183128715F3010130F200BC
:1028B000071A632CF20A0319F30A72087304031946
:1028C000632C6400582C071A6E2CF20A0319F30AC1
:1028D0007208730403196E2C6400632C8312071EA4
:1028E000802C8316C40A0319C50A44084504031939
:1028F000802C12306400FF3E031D7A2C00006E2CE9
:10290000831287117208730403199D2C83164408DF
:102910004504031D8D2C83129D2C450CF100440CA5
:10292000F000F10CF00CF10CF00CF10CF00CF10CCF
:10293000F00C0730F105A12C8312F1017330F00087
:102940008316831283164408F8004508F9008312A1
:102950000034831605118312051583168512831220
:1029600085168316861083128614F1017330F000E9
:102970002808FF3E0318C92C013EE62CF923F92351
:102980008316C301C2017908C1007808C000831210
:10299000C92C3424FF308316E50083126521F80822
:1029A000031DD92C8316C301FF30C200C100C00033
:1029B000831283164008F7004108F8004208F90026
:1029C0004308FA0083128A110A16052F0A108A108A
:1029D0000A158207BE2C0A108A100A158207512F89
:1029E00003300C1EF12C99008316410883120C1E33
:1029F000F72C9900831641088312EE000034FF3F44
:102A000084011F308305073083169F000230990030
:102A100022309800903083129800A001A10110305C
:102A2000A2003030A3008A30A400A501A6012D30F9
:102A3000A700FF30EF00EF106F08831687008312A6
:102A40008714023083169900223098009030831248
:102A5000980002308316990022309800903083123B
:102A600098000F30F70007308101813084000008A2
:102A7000F0390738800064000008F03977048000DE
:102A8000A32564009626412D63000C1E452D990058
:102A90007A2D0530F6007608063C03197A2D8C1A3B
:102AA000532D64004F2D8C1E532D1A088316A00041
:102AB0008312981C612D1A088316A0008312181225
:102AC000181683162008F800831200342808073CE3
:102AD000031D6F2D07300C1E6B2D9900A22D0530A4
:102AE000FC007C08063C0319A22D7C08053C031D54
:102AF0009E2D2830FE006E08F60004300C1E7E2D40
:102B000099006E080C1E822D9900FD016E087D0251
:102B100003189A2D7E08840000088316A0008312F3
:102B20000C1E902D99007E0884000008F606FE0A0F
:102B3000FD0A862D76080C1E9B2D99004F257808DE
:102B4000FC00712D0034B130A8000130EE00662584
:102B50000034F3012830F400F308031DE42D4F2561
:102B60007808F0007008043C0319BA2D4F25780846
:102B7000F000B22D4F257808EE006E08F200F1014A
:102B80006E0871020318D22D7408F5004F257508E0
:102B9000840078088000740884000008F206F40AB3
:102BA000F10AC02D4F257808F206F208031DDF2D2B
:102BB0000130F30006300C1EDB2D9900E32D0530AB
:102BC0000C1EE02D9900AC2D003403306E02003A4B
:102BD0000319502EF1012A08F0007008F1002908AD
:102BE000F0002B30F5000330F4006E087402031877
:102BF000502E7508F50A84000008FA01F2007A08E0
:102C0000F3007508F50A84000008F600F300710867
:102C1000143C03180F2E7108163C03184A2E710835
:102C20001F3C031C4A2EF108031D292E7008033C8B
:102C3000031C292E0310700DF900710DFA0079089C
:102C4000203E8400840A7308800084037208800098
:102C50004A2E700803178D0071088F0072088C00CF
:102C600073088E0083168C170C15831203130B0840
:102C7000F8008B138316031755308D00AA308D0092
:102C80008C14000000008C18432E0C11780883125D
:102C900003138B04F00A0319F10A0230F407F52D2F
:102CA0000730A8000130EE0066250034F0017008FE
:102CB000033C031C8C2EF2017008F1000310700D10
:102CC000F700203E8400840A0008F4008403000812
:102CD000F300700803178D0072088F0073088C00D2
:102CE00074088E0083168C170C15831203130B08BF
:102CF000F8008B138316031755308D00AA308D0012
:102D00008C14000000008C18832E0C11780883129C
:102D100003138B04F00A572E8C2E00342808A900C8
:102D2000FF30A8000230EE0066250034A9252808EF
:102D3000F700313077020319A62E323077020319DB
:102D4000A82E333077020319AA2EAC2EA325AE2E5F
:102D5000E525AE2E5626AE2E8E26AE2E0034FF3F33
:102D6000FF3FFF3FFF3FFF3FFF3FFF3FFF3FFF3F73
:102D7000FF3FFF3FFF3FFF3FFF3FFF3FFF3FFF3F63
:102D8000FF3FFF3FFF3FFF3FFF3FFF3FFF3FFF3F53
:102D9000FF3FFF3FFF3FFF3FFF3FFF3FFF3FFF3F43
:102DA000FF3FFF3FFF3FFF3FFF3FFF3FFF3FFF3F33
:102DB000FF3FFF3FFF3FFF3FFF3FFF3FFF3FFF3F23
:102DC000FF3FFF3FFF3FFF3FFF3FFF3FFF3FFF3F13
:102DD000FF3FFF3FFF3FFF3FFF3FFF3FFF3FFF3F03
:102DE000FF3FFF3FFF3FFF3FFF3FFF3FFF3FFF3FF3
:102DF000FF3FFF3FFF3FFF3FFF3FFF3FFF3FFF3FE3
:102E0000BB308316BF008312A92C7A088316BE003C
:102E10007908BD007808BC007708BB00D030831269
:102E2000A9008316E50183126521F80803191A2FFA
:102E300000301B2F0130AA0083163F08BF0A840010
:102E400000088312AB0083163F08BF0A8400000805
:102E50008312AC0083163F08840000088312AD0083
:102E60000530EF000A126B200A168A150A164E2D3D
:102E70008316C301FF30C200C100C000E501831208
:102E80006521F808031D702F87151E30F700F70B1A
:102E9000472F000087112808FF3E03186B2F013EC3
:102EA000EB2C8316DC01DB014030DA00D901023063
:102EB000DD008312862178081F39FA007708F800B0
:102EC0007A08F9008316C301C2017908C1007808A5
:102ED000C00083126B2FFF308316E500831265213B
:102EE00083164008F7004108F8004208F90043083B
:102EF000FA0083128A110A16822FBB308316BF0094
:102F00008312382F7A088316BE007908BD0078082E
:102F1000BC007708BB00D0308312A9008316E501FE
:102F200083126521F8080319972F0030982F01307C
:102F3000AA0083163F08BF0A840000088312AB0072
:102F400083163F08BF0A840000088312AC00831672
:102F50003F08840000088312AD000530EF000A121C
:102F60006B200A168A150A16562DBB308316BF0031
:102F70008A1583126C288A117A088316BE00790894
:102F8000BD007808BC007708BB00D0308312A900D0
:102F90008316E50183126521F8080319D12F00304B
:102FA000D22F0130AA0083163F08BF0A8400000810
:102FB0008312AB0083163F08BF0A84000008831207
:102FC000AC0083163F08840000088312AD00053072
:102FD000EF000A126B200A168A150A16642D6E0875
:102FE0000C1EF02F99000A1254200A167808063C8D
:102FF000031DF32F00346F2EFF3FFF3FFF3FFF3FC6
:1030000083164014BB30BF0083126F08053C031DBC
:1030100015282D080139003A031D12288316401087
:10302000142883128316401483128316C40183125A
:103030002C088316C30083122B088316C200831248
:103040002A088316C100003040180130C50044082A
:10305000C9004308C8004208C7004108C600450827
:10306000CA008A118312A6228A157A088316BE0026
:103070007908BD007808BC007708BB00D030831207
:10308000A9008316E5018A11831265218A15F808C3
:1030900003194C2800304D280130AA0083163F0840
:1030A000BF0A840000088312AB0083163F08BF0AE2
:1030B000840000088312AC0083163F0884000008D7
:1030C0008312AD000530EF000A128A116B200A1638
:1030D0008A158A150A165D2DFF308316E5008A11C0
:1030E000831265218A15F8080319A4282808FF3ED1
:1030F0000318A428013EC2288316DC01DB01FF303F
:10310000DA00D9000230DD008A11831286218A1587
:103110008316DC01DB014030DA00D9010230DD002A
:103120008A11831286218A1578081F39FA007708D8
:10313000F8007A08F9008316C301C2017908C100BA
:103140007808C0008312A428FF308316E5008A1196
:10315000831265218A15F808031DB5288316C3015B
:10316000FF30C200C100C000831283164008F70080
:103170004108F8004208F9004308FA0083128A1156
:103180000A16BB2F0A108A100A1182077C28BB304E
:103190008316BF008A1183126A228A157A08831661
:1031A000BE007908BD007808BC007708BB00D030AD
:1031B0008312A9008316E5018A11831265218A15FD
:1031C000F8080319E5280030E6280130AA00831624
:1031D0003F08BF0A840000088312AB0083163F0833
:1031E000BF0A840000088312AC0083163F088400E5
:1031F00000088312AD000530EF000A128A116B201F
:103200000A168A158A150A166B2D8316C401FF301B
:10321000E5008A11831265218A15F80803191F2910
:103220008316DC01DB01DA01D9010130DD008A11EE
:10323000831286218A1577088316C40083128316A9
:103240004408F8008312003429308316BD0083122D
:103250002B088316BC0083122A088316BB00831236
:103260002C088316BF0003303F07C000C1008A113D
:103270008312F0248A1583163D088400E030800014
:103280000A128312F7270A1683163D088400831258
:103290002A0880000A12F7270A1683163D088400C0
:1032A00083122B0880000A12F7270A1683163D089E
:1032B000C0003C08C2003B08C100FF30E5008A1195
:1032C000831265218A15F808031986298316410897
:1032D000F70042080F39FA004108C4007A08403864
:1032E000C500C601C7014708DC004608DB004508E9
:1032F000DA004108D9000230DD008A1183128621EC
:103300008A15052178088316C3008312FF308316BF
:10331000E5008A11831265218A15F808031D942996
:10332000FF308316C300831283164308F800400859
:103330008400780880000A128312F7270A160130E9
:103340008316BE003F083E020318B6293D08C000A0
:1033500083120521831640088400780880000A1231
:103360008312F7270A168316BE0AA2298A1183122E
:10337000EF278A158A150A16712D2B088316BD00B2
:1033800083122A088316BC000330BB0083126F0827
:1033900083163B020318232A3D08FA003C08BC0AA6
:1033A0000319BD0ABE007A08BF0029303B0784001C
:1033B0000008C0003F08C2003E08C1004008C3002A
:1033C000FF30E5008A11831265218A15F808031978
:1033D000202A83164108F70042080F39FA004108F5
:1033E000C4007A085038C500C601C7014708DC0090
:1033F0004608DB004508DA004108D9000230DD004C
:103400008A11831286218A15FF308316E5008A11FE
:10341000831265218A1583164308C4006030C500F5
:10342000C601C7014708DC004608DB004508DA0092
:103430004308D9000230DD008A11831286218A15E3
:103440008316BB0AC62907308312A9000130EF009A
:103450000A128A116B200A168A158A150A16772D08
:1034600083164708C8002030C900CA01CB014B08A9
:10347000DC004A08DB004908DA004708D9000230BE
:10348000DD008A11831286218A158316DC01DB0197
:103490004030DA00D9010230DD008A118312862122
:1034A0008A1578088316CA007708C9004A08FA0105
:1034B000F800831200348316C501FF30E5008A113D
:1034C000831265218A15F8080319762A2808FF3E19
:1034D0000318762A013E7D2A83164308C70083120B
:1034E000302278088316C5008312762A8316450891
:1034F000F80083128A150A16CA2A0A108A140A11B9
:1035000082076C2A29308316BD0083122B0883168C
:10351000BC0083122A088316BB0083122C08831672
:10352000BF0003303F07C000C1008A118312F0249E
:103530008A1583163D088400E23080000A12831247
:10354000F7270A1683163D08840083122A08800094
:103550000A12F7270A1683163D08840083122B08E7
:1035600080000A12F7270A168316BE013F083E02A2
:103570000318D62A3D08C0003C08FA003B08BB0AE5
:103580000319BC0AC1007A08C200C4004108C30084
:1035900083125B2A831640088400780880000A1290
:1035A0008312F7270A168316BE0AB62A8A118312D7
:1035B000EF278A158A150A167D2DFF308316E50040
:1035C0008A11831265218A15F8080319292B280806
:1035D000FF3E0318292B013E2C2B83163E08C20008
:1035E0004008C3004108C400C5014408450203184F
:1035F000272B45084207C600C700831230228316D6
:103600004308450784000008C600C700FF30E500F6
:103610008A11831265218A15F8080319242B831651
:103620004708C8003030C900CA01CB014B08DC0094
:103630004A08DB004908DA004708D9000230DD00FB
:103640008A11831286218A158316C50AF52A8312E8
:10365000292B8A150A16472B0A148A140A11820785
:10366000ED2A2B088316BC0083122A088316BB00A0
:10367000033083126F028316BD003C08BF003B0875
:10368000BE002C30C0003D08C1008312DD2A073087
:10369000A9000130EF000A128A116B200A168A1560
:1036A0008A150A16832DFF308316E5008A118312CE
:1036B00065218A15F8080319AF2B2808FF3E031867
:1036C000AF2B013EB22B83164108C7004008C6004D
:1036D0004408C8004508C9004608CB004708CC008C
:1036E0000830CD00CE014E08DC004D08DB00470855
:1036F000DA004608D9000330DD008A1183128621E2
:103700008A158316DC010930DB00DA01D9010330A8
:10371000DD008A11831286218A158316CA014908A1
:103720004A020318AD2B4808C80AC80ACB00DC01BE
:103730000930DB00DA01D9010330DD008A11831280
:1037400086218A1583164B08840077088000840A36
:10375000780880000230CA078F2B8312AF2B8A159E
:103760000A16D92B0A148A140A118207632B8316AE
:10377000BF0183122C088316BE0083122B08831608
:10378000BD0083122A088316BC0083122D08EF00A7
:1037900083163F08C3003E08C2003D08C1003C0834
:1037A000C0002D30C40083126F088316C500831239
:1037B000532BC430A9000430EF070A128A116B2082
:1037C0000A168A158A150A16892DFF308316E50018
:1037D0008A11831265218A15F80803193C2C2808E0
:1037E000FF3E03183C2C013E3F2C83164208C800C4
:1037F0004108C7004508C9004608CA004708CC0070
:103800004808CD000830CE00CF014F08DC004E083C
:10381000DB004808DA004708D9000330DD008A11D0
:10382000831286218A158316CB014A084B0203189E
:103830003A2C4908C90AC90A8400840A0008FA0017
:1038400084030008CC007A08CD000A30CE00CF01F6
:103850004F08DC004E08DB004D08DA004C08D900A8
:103860000330DD008A11831286218A150230831607
:10387000CB07152C83123C2C8A150A16652C0A10CE
:103880008A100A158207F52B8316BF0183122C08B4
:103890008316BE0083122B088316BD0083122A08EC
:1038A0008316BC00043083126F028316C0003F08E9
:1038B000C4003E08C3003D08C2003C08C1002D30D2
:1038C000C5004008C6008312E52B0730A90001306F
:1038D000EF000A128A116B200A168A158A150A1639
:1038E0008F2D2A308316BB0097308312A9008316D0
:1038F0003B08BC008A11831234248A1583163C08C5
:103900008400840A790880008403780880000330EA
:103910008312EF000A128A116B200A168A158A1583
:103920000A16952D2A308316BB0083122C08EF004F
:1039300083163B088400840A0008BD008403000845
:10394000BC003D08BF003C08BE002C30C000831204
:103950006F088316C100E6308312A9000330EF0719
:103960000A128A116B200A168A158A150A169B2DCF
:103970002A308316BB003B088400840A0008BD007F
:1039800084030008BC00033083126F028316BE005C
:103990003D08C0003C08BF002C30C1003E08C200FA
:1039A00007308312A9000130EF000A128A116B2040
:1039B0000A168A158A150A16A12D8316BB013B0823
:1039C000033C031C2F2DBD013B08BC0003103B0D25
:1039D000F700BE003E0A0A128A11831235200A1629
:1039E0008A15FA0083163E080A128A1183123520BE
:1039F0000A168A158316BF007A08C0003C08831295
:103A000003178D00831603133D08831203178F00DD
:103A1000831603133F08831203178C0083160313C6
:103A20004008831203178E0083168C170C1583121F
:103A300003130B08F8008B138316031755308D0002
:103A4000AA308D008C14000000008C18252D0C115C
:103A50007808831203138B048316BB0ADF2C8A01B8
:103A6000831282018A150A16A72D2908AA00FF30A1
:103A7000A9000230EF000A128A116B200A168A157B
:103A80008A150A16A92D8316BA08031DAA2D8312BA
:103A90002908523C031D502D8A11002F8A15A92D8B
:103AA0002908533C031D582D8A117D2F8A15A92DF5
:103AB0002908543C031D5E2D0028A92D2908553CDA
:103AC000031D662D8A11B52F8A15A92D2908563C8C
:103AD000031D6C2DC728A92D2908603C031D722DDC
:103AE0002429A92D2908613C031D782DBD29A92D64
:103AF0002908623C031D7E2D822AA92D2908633CDA
:103B0000031D842D312BA92D2908653C031D8A2D09
:103B1000B72BA92D2908643C031D902D442CA92DF9
:103B20002908663C031D962D712CA92D2908673C98
:103B3000031D9C2D922CA92D2908683C031DA22D44
:103B4000B82CA92D2908313C031DA82DDD2CA92D49
:103B5000352D831683128A150A161D2E84011F30F7
:103B60008305073083169F000230990022309800A9
:103B7000903083129800023083169900223098000A
:103B800090308312980002308316990022309800FA
:103B900090308312980002308316990022309800EA
:103BA00090308312980002308316990022309800DA
:103BB0009030831298007330F000F10174100714F4
:103BC0000714993083168700103086000B3085006B
:103BD000B530831290008F018E0183160C14C03013
:103BE00083128B040F30F70007308101813084008D
:103BF0000008F0390738800064000008F0397704C5
:103C000080000A128A114B200A168A150A128A119C
:103C1000B4200A168A150B138B138B1B0C2E8316DC
:103C20000C108312061564008A1166288A1578081C
:103C30008316B900BA008312432D132E63001E2E83
:103C40000C117808831203138B048316B20AD82D43
:103C50008A01831282018A150A16A62E2908AA0053
:103C6000FF30A9000230EF000A128A116B200A16F9
:103C70008A158A150A16A82E8316B108031DA92EC7
:103C800083122908523C031D492E8A11862A8A155F
:103C9000A82E2908533C031D512E8A11142B8A1576
:103CA000A82E2908543C031D592E8A11DF2B8A1592
:103CB000A82E2908553C031D612E8A11AB2C8A15AC
:103CC000A82E2908563C031D692E8A11002F8A153B
:103CD000A82E2908603C031D712E8A119A2F8A157F
:103CE000A82E2908613C031D772EC929A82E290872
:103CF000623C031D7D2E522AA82E2908633C031D19
:103D0000832E132BA82E2908653C031D892EAD2B6D
:103D1000A82E2908643C031D8F2E4E2CA82E29089E
:103D2000663C031D952E7B2CA82E2908673C031D9D
:103D30009B2E152DA82E2908683C031DA12EB02D01
:103D4000A82E2908313C031DA72ED62DA82E2E2ED5
:103D5000831683128A150A161C2F84011F308305CF
:103D6000073083169F00023099002230980090306F
:103D70008312980002308316990022309800903008
:103D800083129800023083169900223098009030F8
:103D900083129800023083169900223098009030E8
:103DA00083129800023083169900223098009030D8
:103DB000831298007330F000F101F4100714071417
:103DC000993083168700103086000B308500B5309F
:103DD000831290008F018E0183160C14C030831261
:103DE0008B040F30F7000730810181308400000818
:103DF000F0390738800064000008F039770480004B
:103E00000A128A114B200A168A150A128A11B42046
:103E10000A168A150B138B138B1B0B2F83160C1092
:103E20008312061564008A1100288A157808831603
:103E3000B000B10083123C2E122F63000319912FA2
:103E4000313077020319932F952F0A128A11AE2071
:103E50000A168A15962F0A128A11D7200A168A1571
:103E6000962F0A128A113F210A168A15962F0A12D6
:103E70008A11CC210A168A15962F0A128A119821C6
:103E80000A168A15962F0A128A11E4210A168A1533
:103E9000962F0A128A1124220A168A15962F0A12C0
:103EA0008A1184220A168A15962F0A128A119422E0
:103EB0000A168A15962F0A128A11C4220A168A1522
:103EC000962F0A122B220A16962F0A1222230A165E
:103ED000962F0A128B240A16962F0A120B260A1600
:103EE000962F8A113E208A15962F0A128A11F127E1
:103EF0000A168A15962F0A12C9270A16962F8A11B2
:103F000000278A15962F0020962F8E20962FD920D5
:103F1000962F7D21962F3A22962FBE22962F52233E
:103F2000962FE123962F5A24962FAE245A2E630003
:103F3000220803178C000313210803178E00831631
:103F400003178C170C158B1355308D00AA308D007C
:103F50008C140000FF3EFF3EFF3EFF3EFF3EFF3E53
:103F6000FF3EFF3EFF3EFF3EFF3EFF3EFF3EFF3E69
:103F7000FF3EFF3EFF3EFF3E0C118C1383016400A9
:103F80000D1EBF2F0D1283168101831269080317BE
:103F90008D000313680803178F00DC2783120317B3
:103FA0000C080313A20003170E080313A100080056
:103FB000E90A0319E80A0800831603178C170C1482
:103FC0000000FF3EFF3E8C138301080021081F39CB
:103FD000E8001F3A031968122208E900C627462E96
:103FE00068081E391E3A0319FC2F6808031DFB2FB1
:103FF0006908C039031D8B27D827462EFF3FFF3F96
:104200000200FF00FF00FF00FF00FF00FF00FF00B3
:10421000FF00FF00FF00FF00FF00FF00FF00FF00A6
:10422000FF00FF00FF00FF00FF00FF00FF00FF0096
:10423000FF00FF00FF00FF00FF00FF00FF00FF0086
:10424000FF00FF00FF00FF00FF00FF00FF00FF0076
:10425000FF00FF00FF00FF00FF00FF00FF00FF0066
:10426000FF00FF00FF00FF00FF00FF00FF00FF0056
:10427000FF00FF00FF00FF00FF00FF00FF00FF0046
:10428000FF00FF00FF00FF00FF00FF00FF00FF0036
:10429000FF00FF00FF00FF00FF00FF00FF00FF0026
:1042A000FF00FF00FF00FF00FF00FF00FF00FF0016
:1042B000FF00FF00FF00FF00FF00FF00FF00FF0006
:1042C000FF00FF00FF00FF00FF00FF00FF00FF00F6
:1042D000FF00FF00FF00FF00FF00FF00FF00FF00E6
:1042E000FF00FF00FF00FF00FF00FF00FF00FF00D6
:1042F000FF00FF00FF00FF00FF00FF00FF00FF00C6
:10430000FF00FF00FF00FF00FF00FF00FF00FF00B5
:10431000FF00FF00FF00FF00FF00FF00FF00FF00A5
:10432000FF00FF00FF00FF00FF00FF00FF00FF0095
:10433000FF00FF00FF00FF00FF00FF00FF00FF0085
:10434000FF00FF00FF00FF00FF00FF00FF00FF0075
:10435000FF00FF00FF00FF00FF00FF00FF00FF0065
:10436000FF00FF00FF00FF00FF00FF00FF00FF0055
:10437000FF00FF00FF00FF00FF00FF00FF00FF0045
:10438000FF00FF00FF00FF00FF00FF00FF00FF0035
:10439000FF00FF00FF00FF00FF00FF00FF00FF0025
:1043A000FF00FF00FF00FF00FF00FF00FF00FF0015
:1043B000FF00FF00FF00FF00FF00FF00FF00FF0005
:1043C000FF00FF00FF00FF00FF00FF00FF00FF00F5
:1043D000FF00FF00FF00FF00FF00FF00FF00FF00E5
:1043E000FF00FF00FF00FF00FF00FF00FF00FF00D5
:1043F000FF00FF00FF00FF00FF00FF00FF00FF00C5
:08400000FF3FFF3FFF3FFF3FC0
:00000001FF
